:1000000001308A00A1290000D3346D38EC32202A57
:10001000E832F236EF36653AE8327210A0060A008E
:10002000CC224410253658100D050000D63C7336FE
:100030006532EE3220265321A0126C2CA0060A0055
:10004000A013200883168700831287130830F80056
:1000500029280000F8173A28F813AF0C031887175F
:10006000031C871378173A287813F80B2D283828A3
:10007000000087173F308400840B3C280000F81BE9
:100080002C28781B34280800831603178C170C14AF
:100090000000000083120C087F390319882803131D
:1000A000AB0003170D080313AC0003170F0803136D
:1000B000AD002B08AF0020202C0803178D00031380
:1000C0002D0803178F0083168C170C1400000000F6
:1000D00083120C0D0E0D7F39031988280313AB0012
:1000E00003170D080313AC0003170F080313AD002B
:1000F0002B08AF0020202C0803178D0003132D08B8
:1001000003178F008D0A03198F0A0313442803175E
:1001100003138A110A120D2A0830F8000000871113
:10012000A01120088316870000008312AB0D071270
:10013000031CA0282016200883168700A4288312F9
:10014000201220088316870000008312A0152008C3
:10015000831687008312871DAB28F80B8E280000BA
:100160008711A01120088316870000008312201633
:10017000200883168700000000008312A0152008C5
:10018000831687008312871DC328F8010000071A11
:1001900078148711A0112008831687008312071294
:1001A0002012200883168700831208002B30840059
:1001B000831300080319E9280230F800F701F70B50
:1001C000DF28F80BDE289730F700F70BE528800BC7
:1001D000DC2808000830AC007708AD0020162008A5
:1001E0008316870000008312A0152008831687005D
:1001F0008312871DF928071A0314071E0310F80D30
:100200000000A01120088316870083128711AC0B11
:10021000EE2820162008831687000000831207129C
:100220002D0803191829201220088316870083122D
:100230000000A0152008831687008312871D1E2941
:1002400000008711A0112008831687000000831288
:100250000712201220088316870083128A110A12BF
:10026000572B831603178C170C140000000003187B
:10027000602983120C087F390313AC0003170D08A3
:100280000313AD0003170F080313AE002C08AF00D3
:1002900020202D0803178D0003132E0803178F004D
:1002A00083168C170C140000000083120313AB0B91
:1002B0005A295D298316031760297F29831603179E
:1002C00083120C0D0E0D7F390313AC0003170D08BC
:1002D0000313AD0003170F080313AE002C08AF0083
:1002E00020202D0803178D0003132E0803178F00FD
:1002F0008D0A03198F0A03100313AB0B3129080071
:10030000AC1B92290F30F7002B0EF7050A3077024D
:1003100003188D293030F7078F292C08F707770845
:10032000AF0020200F30AB050A302B0203189A29AA
:1003300030309C29AC132C08AB072B08AF002020D1
:100340000800840183131F308305713083168F00EA
:100350000F088312A01320088316870083128717C3
:10036000831603170908C039890003131F129F124F
:100370000030031788008312870188018901FF304C
:100380000313A000831603170908C039890003135B
:100390001F129F12003003178800831203131F13CC
:1003A0009F1383169F1383121F149412A012200808
:1003B0008316870083122016200883168700831275
:1003C000A0112008831687000130831294000030AA
:1003D000831694000108C739083881008312900100
:1003E0000030F8009200003083169200831220152E
:1003F0002008831687008312970183169B019C01B6
:1004000001309D00831203178701880189010430A0
:100410008D0000308F0003134428A701A901201686
:1004200020088316870000008312A0152008831679
:10043000870000008312071220122008831687000D
:10044000000083128711A011200883168700AA30AC
:100450008312AB008C206130AB008C20201620086A
:100460008316870000008312A015200883168700DA
:1004700000008312871D3A2A0712201220088316D3
:100480008700000083128711A011200883168700BF
:10049000AA308312AB008C20AB018C2020122008E4
:1004A0008316870000008312A0152008831687009A
:1004B0008312871D592A00005D2A0000201620089B
:1004C00083168700000001308312AB00D62020166F
:1004D00020088316870000008312A01520088316C9
:1004E000870000008312071220122008831687005D
:1004F000000083128711A011200883168700AA30FC
:100500008312AB008C203E30AB008C2020162008DC
:100510008316870000008312A01520088316870029
:1005200000008312871D922A0712201220088316CA
:100530008700000083128711A0112008831687000E
:10054000AA308312AB008C204030AB008C202012EC
:1005500020088316870000008312A0152008831648
:1005600087008312871DB22A0000B62A00002016D9
:10057000200883168700000001308312AB00D620CC
:10058000201620088316870000008312A01520087B
:10059000831687000000831207122012200883169A
:1005A0008700000083128711A0112008831687009E
:1005B000AA308312AB008C203F30AB008C20201679
:1005C00020088316870000008312A01520088316D8
:1005D000870000008312871DEB2A071220122008D3
:1005E00083168700000083128711A011200883164C
:1005F0008700AA308312AB008C20AB018C20201224
:1006000020088316870000008312A0152008831697
:1006100087008312871D0A2B00000E2B0000201676
:10062000200883168700000001308312AB00D6201B
:10063000201620088316870000008312A0152008CA
:1006400083168700000083120712201220088316E9
:100650008700000083128711A011200883168700ED
:10066000AA308312AB008C204430AB008C202016C3
:1006700020088316870000008312A0152008831627
:10068000870000008312871D432B071220122008C9
:1006900083168700000083128711A011200883169B
:1006A0008700AB308312AB008C20F701EA28780872
:1006B000A800201220088316870000008312A015CE
:1006C0002008831687008312871D642B0000682B87
:1006D00000002016200883168700000001308312D6
:1006E000AB00D620103003178D0000308F000310B0
:1006F00004300313AB0031212808AB003730AC00C5
:1007000080212030AF0020200D30AF0020200A30A3
:10071000AF0020202808733C031DAA2B0130A7023C
:10072000163003178D0000308F0003100D300313B7
:10073000AB0031212708AB003730AC0080212030DE
:10074000AF0020200D30AF0020200A30AF00202065
:10075000A82B5C2C2016200883168700000083122B
:10076000A0152008831687000000831207122012AC
:10077000200883168700000083128711A01120082B
:1007800083168700AA308312AB008C204430AB0064
:100790008C20201620088316870000008312A015E5
:1007A00020088316870000008312871DD52B0712AF
:1007B0002012200883168700000083128711A011E1
:1007C000200883168700AA308312AB008C20733078
:1007D000AB008C20201220088316870000008312B3
:1007E000A0152008831687008312871DF52B0000B3
:1007F000F92B0000201620088316870000004030E7
:100800008312AA00A401A301A601A50120162008B5
:100810008316870000008312A01520088316870026
:1008200000008312071220122008831687000000A0
:1008300083128711A011200883168700AA30831223
:10084000AB008C206030AB008C2020162008831673
:10085000870000008312A01520088316870000007F
:100860008312871D312C071220122008831687005F
:10087000000083128711A011200883168700AA3078
:100880008312AB008C202708AB008C20201220089C
:100890008316870000008312A015200883168700A6
:1008A0008312871D512C0000552C000020162008B3
:1008B00083168700000083120130A7076430AB0065
:0608C000D6200F2A6300A0
:04400E00F52CFF3F4F
:00000001FF
